:100000005EC043C377C076C075C074C073C072C091
:1000100071C070C06FC06EC06DC06CC06BC0050198
:100020000905A1010901A1000930093115002502C6
:10003000750295028102C0050919012904150025E0
:1000400001750195048102C00403090416037600BA
:1000500069006B006900740073002E0063006F007C
:100060006D00280355005300420020004E0045005B
:100070005300200050006100640020006100640013
:100080006100700074006500720012011001000030
:100090000008EA1D07100001010200010902220008
:1000A0000101008032090400000103000000092161
:1000B00001010001222A000705810308000A11241A
:1000C0001FBECFE5D2E0DEBFCDBF10E0A0E6B0E0BE
:1000D000E6E7F9E002C005900D92A236B107D9F724
:1000E00010E0A2E6B0E001C01D92AB39B107E1F724
:1000F00056D03FC485CF80E00895AF92BF92DF9283
:10010000EF92FF920F931F93CF93DF9308E010E0DD
:10011000EE2480E8F82EDF2CDE0CD1BEA3D2A82E70
:10012000E5015E01B92EE50199E0C433D9070CF46D
:10013000ED2CF6940150104071F78E2D815081BF47
:1001400081B70E2D10E00F5F1F4F90E008171907C1
:1001500074F416C08C179D0714F4E1B6EC0181B756
:100160008F5F81BF81B790E0081719074CF07AD2F2
:100170008453994097FFEECF909581959F4FEACF9A
:10018000E1BE61B780E090E0E6D3DF91CF911F91AF
:100190000F91FF90EF90DF90BF90AF9008950F9375
:1001A0001F93E199FECF80E090E0CDD38F3F09F01F
:1001B00081BF81E291EA0197F1F700C00000479A00
:1001C000B89A8FE49DE2A9E181509040A040E1F708
:1001D00000C00000B8982EE088E190E00FB6F894D7
:1001E000A89581BD0FBE21BD17D27894BB9AB9984E
:1001F000BC9AC398C49815E005E2A895CFD0809129
:10020000700084FFFACF10936400C49A95E09A9529
:10021000F1F700C0C498A5E0AA95F1F700C0B19924
:1002200002C000936400C39AB5E0BA95F1F700C02C
:10023000C39885E08A95F1F700C0B19905C0809117
:100240006400806180936400C39A95E09A95F1F709
:1002500000C0C398A5E0AA95F1F700C0B19905C008
:1002600080916400806480936400C39AB5E0BA957D
:10027000F1F700C0C39885E08A95F1F700C0B19905
:1002800005C080916400806880936400C39A95E003
:100290009A95F1F700C0C398A5E0AA95F1F700C0C0
:1002A000B1990DC090916400892F869586958D5FD8
:1002B0008370880F880F937F982B90936400C39A64
:1002C000B5E0BA95F1F700C0C39885E08A95F1F7DB
:1002D00000C0B1990DC090916400892F86958695D4
:1002E0008F5F8370880F880F937F982B90936400A3
:1002F000C39A95E09A95F1F700C0C398A5E0AA9536
:10030000F1F700C0B19909C080916400982F9D5FFA
:1003100093708C7F892B80936400C39AB5E0BA9563
:10032000F1F700C0C39885E08A95F1F700C0B19954
:1003300009C080916400982F9F5F93708C7F892BF8
:100340008093640084E690E061E001D056CF1F9373
:10035000162F2091700024FF1DC02091710038E8F5
:10036000232720937100A82FB92F812F815090E06F
:100370008D589F4FE2E7F0E02D912193E817F907A0
:10038000D9F782E790E0612F69D11C5F109370006C
:100390001F9108952AE520937000E5CF1F93CF9316
:1003A000DF9380918100835087FD09C020917E00FA
:1003B00090917D009D3209F45DC010928100809182
:1003C000600084FF39C0609161006F3FA9F169301E
:1003D00008F47DC06850609361008091650098E8E2
:1003E0008927809365001CE068E020917F003091B0
:1003F00080008091620086FF80C0462F415050E00F
:10040000CA0189599F4FF901A6E6B0E074917D9326
:100410003196A817B907D1F74F5F5F4F420F531FAF
:100420005093800040937F0086E690E017D11C3007
:1004300009F05DC01093600094E186B3857099F473
:100440009150D9F71092820010927C0011E08091B7
:100450006300181721F0112359F010936300DF9106
:10046000CF911F91089511E0992389F310E0EFCF08
:1004700044DEF3CF883009F0A0CFCCE0D0E0C21B3F
:10048000D109CB57DF4F83EC809365008AE58093D9
:1004900060001092620088818076F1F59A81109256
:1004A0006E0089818823D9F510926F002EE630E026
:1004B00082E03093800020937F009F81992321F474
:1004C0009E81981708F4892F8093610076CF10924F
:1004D00061008091650098E8892780936500662314
:1004E00009F082C086E690E060E0B8D014E08FEFBB
:1004F00080936100109360009FCFD901462F415037
:1005000050E0CA0189599F4FE6E6F0E07D91719372
:10051000E817F907D9F780CFCE01EDDDCECF8530D2
:1005200071F0863091F0883001F1893011F18A3014
:1005300071F18B3081F12EE630E080E0BACF9093FC
:1005400082002EE630E080E0B4CF8B818130B9F0BC
:10055000823091F1833031F18132F1F18232A1F1B7
:1005600080E090E490936200A8CF24E830E081E03E
:10057000A0CF909384002EE630E080E09ACF8AE806
:1005800090E09093800080937F0082E1EACF2EE696
:1005900030E081E08ECF8BE4809371002EE630E076
:1005A00080E087CF992319F588E490E0909380004C
:1005B00080937F0084E0D5CF8CE990E09093800019
:1005C00080937F0082E2CDCF8EE190E09093800017
:1005D00080937F008AE2C5CF8EEA90E090938000FE
:1005E00080937F0089E0BDCF162F1C5FFECE913037
:1005F00059F0923009F0B4CF82E690E090938000F9
:1006000080937F0088E2ADCF8CE490E090938000EF
:1006100080937F0086E1A5CF85B7836085BF8BB7C8
:1006200080648BBF8BE4809371008AE580937000B7
:100630000895A82FB92F80E090E041E050EA60953E
:1006400030E009C02D9182279795879510F0842777
:100650009527305EC8F36F5FA8F30895EADF8D93A6
:100660009D930895A6E088279927AA9569F0019798
:10067000E1F3B099FCCFB09BFECF81E09927A6B300
:10068000019611F0A570D9F70895CF93CFB7CF9306
:10069000C395B09BE9F7B09B0BC0B09B09C0B09B62
:1006A00007C0B09B05C0B09B03C0B09B01C0D5C0C4
:1006B0000F92DF93C0917E00DD27CB57DF4F012ED5
:1006C000B09B03C0DF910F90E6CF2F930F931F9342
:1006D0004F932FEF4F6F06B300FB20F95F933F93CB
:1006E00050E03BE065C016B30126502950FDC89587
:1006F00056B3012700FB25F92F7306B3B1F050273D
:10070000102710FB26F906B22230F0F000C016B315
:10071000012700FB27F90126502906B22430E8F50D
:100720004F77206816B30000F6CF50274F7D206228
:1007300006B2102F000000C006B300265029102773
:1007400010FB26F906B2E2CF4F7B06B3206400C04F
:10075000DACF01265029157006B269F14E7F21606B
:10076000012F16B328C0002650294D7F06B2226003
:10077000102F29C0012650294B7F06B22460012F7B
:100780002DC016B301265029477F2860000006B20D
:100790002EC04F7E06B3206130C0422706B3499376
:1007A00000265029102706B24FEF10FB20F9297FB1
:1007B00016B379F2157059F10126502906B20127B6
:1007C00000FB21F9237F06B371F200265029315036
:1007D000D0F006B2102710FB22F9277E16B351F293
:1007E00001265029012700FB06B223F92F7C49F28C
:1007F000000006B3102710FB24F90026502906B28A
:100800002F7939F270CF10E41ABF002719C03B507E
:100810003195C31BD04010E41ABF0881033C09F195
:100820000B34F9F020917C001981110F1213EDCFD8
:100830004A81441F093651F10D3211F0013E29F76A
:10084000009383003F915F914F911F910F912F91E2
:10085000DF910F90CAB7C6FD1BCFCF91CFBFCF910D
:10086000189520918300222369F3109181001123B0
:1008700079F534307AF13093810020937D00109126
:100880007E003BE0311B30937E0024C0009181004C
:100890000130F4F40AE54F7049F43091600034FD02
:1008A0001AC000936000C5E6D0E019C03091700016
:1008B00034FD11C000937000C1E7D0E010C00527DF
:1008C00010E000C021C0052710E0C89508BB14C087
:1008D0003AE501C032ED032EC0E0D0E032E017B3BC
:1008E0001560C09A08B317BB55E020E84FEF20FF12
:1008F000052708BB279517951C3F28F70000455290
:10090000B0F720FF0527279508BB17951C3FB8F6C1
:1009100029913A9561F70A7F10918200110F08BB67
:10092000C250D04011F010937C0010E41ABF016057
:1009300017B31A7F402F4A7F54E05A95F1F708BB4E
:1009400017BB48BB7FCFE199FECF9FBB8EBBE09A20
:1009500099278DB30895262FE199FECF1CBA9FBB2E
:100960008EBB2DBB0FB6F894E29AE19A0FBE0196AA
:060970000895F894FFCF8A
:020976005AFF26
:00000001FF
